:020000002B28AB
:100008003F288A0182002F34433431344734313455
:100018000D3400344F344B340D3400348A014A080F
:10002800CA0A82002F341934003447341C3400348F
:1000380031341F34003450346A2852346C28563412
:1000480062282E345F280D34562800340034831675
:100058002430850050309F00961683128B1514307B
:10006800C9006F208B13CF1A8A2005080B108B1735
:100078000A309520352828211630CA004D21D00095
:100088001220003A03195028500603194D28CA0AAD
:1000980044281220CA0042281220003A031D35289D
:1000A8003F30E5205A2065201E2135280D30E528EF
:1000B8001F305A2041282E30E52056286630C220AD
:1000C800562805160A30952005120800AC20C900EC
:1000D8004908C2205628CF127C20051D7728051212
:1000E8000A30C80008000516C80B0800CF1608001B
:1000F8004908C5008514842085108420C50B7E28F6
:1001080000000630C700C70B872808000730D92031
:1001180014308F200800C40064309520C40B902848
:100128000800C300A020C30B962808000230A128AD
:100138000A30A1281430A128C830C20000000000ED
:1001480000000000000000000000C20BA228080008
:10015800D2014D21C7003030C702031CC0280A3025
:1001680047020318C0280310D20D5208D20DD20D31
:10017800D2074708D207AD28520808004F12CC0012
:100188006430CA200A30CA204F160130CD00303002
:10019800CE004D08CC02031CD428CE0A4F16CE2818
:1001A800CC074E084F1AE52008000000E90069084E
:1001B800E90A0520C700003A031908004708E520A6
:1001C800DB28C70054305307D30A8400470880004F
:1001D8000D3A031D0800D30102290330EA00FB2071
:1001E800CF180800C8309520EA0BF3280800022130
:1001F80054082F3A03192629CF14080054308400D4
:1002080006291A21F101851E05299C20F10B0729D1
:10021800851E0529831685128312000855210008BA
:10022800840A0D3A031D1129D30108001E213F3904
:10023800013EA1286B08EC076C08ED076D08EB0E72
:10024800EB070800CF152929CF11CF10DE010030A8
:10025800EF006430EE009E2072214F1954284F1889
:100268003C29EE0B2F29CF190800EF0B2F29080086
:10027800C7005E08093A031935285F305E07DE0AB1
:100288008400470880000D3A031D2B29CF14DE0196
:1002980008005F305E07DE0A840000080800DE03FD
:1002A8000800D20083168512831206306A210230B4
:1002B8006A210830C5000130D20D031803306A21C5
:1002C800C50B5F298316851683120800C7009E2078
:1002D80085129E20C70B6D29851608004F114F10F7
:1002E800851A08008E2103198C298E2103198C295F
:1002F800D1000830C500D2018E2103198C29C7000E
:100308005108C702D20DC50B802952084F140800A6
:100318004F150800C701C70A031908000A30F20080
:10032800F20B9429851A8F29C701C70A03190800F7
:100338000A30F200F20B9E294708851E9929080009
:02400E00E400CC
:00000001FF
